:1000000000308A0085280000FF00030E8301A10054
:100010007F08A0000A08A8008A01A00E0408A20018
:100020007708A3007808A4007908A5007A08A6003C
:100030007B08A700831383120B1E20288B183328FC
:10004000220884002308F7002408F8002508F90096
:100050002608FA002708FB0028088A00210E8300E2
:10006000FF0E7F0E09008030B500FA012908B600A6
:10007000B5080319492886183B28360835050319A1
:100080004328061544280611861C44280310B50C85
:1000900038288B108A112028F801F901F701FA019C
:1000A0003308031D56283208031970281030B40095
:1000B0000310B00DB10DF70DFA0D33087A02031DD0
:1000C000632832087702031C6C283208F702031CED
:1000D000FA033308FA020314F80DF90DB40B58288B
:1000E0000000D5282E30840000080319842806302B
:1000F000F800F701F70B7A28F80B79287B30F70026
:10010000F70B8028800B7728E72884011F308305B0
:1001100007309F00AA01A901303065000330660056
:10012000A53090008316011383120B16C0308B0488
:100130008F018E01AB012B08C73C031CB12885142D
:1001400005111230F700F70BA32800000000051579
:1001500085101230F700F70BAB2800000000AB0A47
:100160009B280511AD01AC012D08073C031CE428B8
:10017000031DBE282C08CF3C031CE428051ADA28EE
:100180000F08FA000E08F7000F087A02031DC028B6
:100190007708AE007A08AF002F08B1002E08B00033
:1001A0000130B3002430B2004C287908AA00780846
:1001B000A900E4283130F700F70BDC28000000002C
:1001C000AC0A0319AD0AB4283230AE007228982860
:0601D0000030F80063009E
:02400E006A3F07
:00000001FF
